:100000000C94E0000C949C080C94C9080C94080112
:100010000C9408010C9408010C9408010C9408013C
:100020000C9408010C9408010C9408010C9408012C
:100030000C9408010C9408010C9408010C9408011C
:100040000C94F6080C9408010C94930A0C94C50ABD
:100050000C9408010C9408010C9408010C940801FC
:100060000C9408010C940801000000080002010033
:100070000003040700000000000000000102040863
:100080001020408001020408102001020408102002
:10009000040404040404040402020202020203032E
:1000A00003030303000000002300260029000000D2
:1000B0000000250028002B0000000000240027007D
:1000C0002A0000407A10F35A00A0724E180900105E
:1000D000A5D4E80000E87648170000E40B540200BD
:1000E00000CA9A3B000000E1F505000080969800E8
:1000F000000040420F000000A08601000000102711
:1001000000000000E80300000000640000000000A0
:100110000A00000000000100000000002C76D888D2
:10012000DC674F0823DFC1DFAE59E1B1B796E5E3E5
:10013000E453C63AE651997696E8E6C28426EB89FE
:100140008C9B62ED407C6FFCEFBC9C9F40F2BAA59B
:100150006FA5F490055A2AF75C936B6CF9676DC133
:100160001BFCE0E40D47FEF520E6B500D0ED902E37
:100170000300943577050080841E080000204E0A95
:10018000000000C80C333333330F986E12831141D3
:10019000EF8D2114893BE65516CFFEE6DB18D1849E
:1001A0004B381BF77C1D901DA4BBE42420328472C5
:1001B0005E228100C9F124ECA1E53D274101F50A49
:1001C00011241FBECFEFD8E0DEBFCDBF11E0A0E00D
:1001D000B1E0E2ECF3E202C005900D92AC34B1075D
:1001E000D9F722E0ACE4B1E001C01D92A036B2071D
:1001F000E1F711E0C0ECD1E004C02297FE010E94BB
:10020000930CCC3BD107C9F70E94390B0C94DF113A
:100210000C94000061E081E10E94FB0960E081E153
:100220000E94340A61E089E00E94FB0960E083E0FB
:100230000C94FB091F93CF93DF93182FEB0161E020
:100240000E94340ABE01882777FD8095982F0E946E
:100250006F0960E0812FDF91CF911F910C94340AD8
:1002600060E089E00E94340A83B7817F846083BFA5
:1002700083B7816083BF7894889583B78E7F83BF6F
:10028000089520E042E06AE086E591E00C94770270
:10029000CF92DF92EF92FF920F931F93CF93DF9352
:1002A000CDB7DEB7EC970FB6F894DEBF0FBECDBF6B
:1002B00029E288E190E00FB6F894A8958093600059
:1002C0000FBE2093600083E00E946A0A909365014C
:1002D00080936401019709F069C061E089E00E94A0
:1002E000340A64E670E080E090E00E946F0920E04C
:1002F00042E050E06BE586E591E00E94030561E095
:1003000086E591E00E94200866E071E086E591E0D4
:100310000E94BE0460E086E591E00E945A087E01DA
:1003200023E3E20EF11C682F70E080E090E00E9471
:10033000540C870123E043E00E94970C80914E010A
:100340009E012F5F3F4F690181110EC0F90101909D
:100350000020E9F73197E21BF30BF0934D01E09396
:100360004C0181E080934E01FF92EF9287E191E092
:100370009F938F93DF92CF920E94B80C8EE1E82E6C
:1003800002E020914C01A60161E070E086E591E079
:100390000E94A70264E670E081E10E941A010F90BA
:1003A0000F900F900F900F900F9002C00E9430019D
:1003B000EC960FB6F894DEBF0FBECDBFDF91CF91A4
:1003C0001F910F91FF90EF90DF90CF900895CF9302
:1003D000CFB7F89480916901811127C0EAE9F0E074
:1003E0008491E6E8F0E09491E82FF0E0EE0FFF1F33
:1003F000E854FF4FA591B4918C91892321F461E0D9
:100400008AE00E94340A61E08AE00E94FB098CB510
:1004100080618CBD8CB580648CBD61E08DE00E94F4
:10042000FB0961E08BE00E94FB09809169018F5F0D
:1004300080936901CFBFCF910895089581E08093A3
:100440006C010895CF93DF93EC0161E08A810E94F3
:10045000340A80916801882361F09FB7F894209155
:10046000680180916601213019F48DBB9FBF01C0E6
:100470008FBF8A858CBD8B858DBDDF91CF9108950F
:10048000FC018CB582878DB5838734852585809165
:100490006801882399F09FB7F894809168018130B2
:1004A00059F48DB3809366014DB3809167018095B7
:1004B00084238DBB9FBF02C0909366013CBD2DBDC0
:1004C0008CB5837F8CBD8CB58F7D8CBD8CB58C7FBE
:1004D0008CBD8DB58E7F8DBD60E082810C94340A19
:1004E0008EBD00000DB407FEFDCF8EB50895FC0152
:1004F00081E291E09183808380E5848781E0858734
:10050000628343838093770117828FE180872187FD
:100510000895CF93DF93EB01DC01ED91FC91048012
:10052000F581E02D0995882371F0809174019091F7
:1005300075018C179D0711F0CD2B29F481E0909166
:100540006F01911101C080E0DF91CF9108952F924A
:100550003F924F925F926F927F928F929F92AF9253
:10056000BF92CF92DF92EF92FF920F931F93CF93A0
:10057000DF93EC015B014A01722E602E10E0CE2C5D
:10058000D12CE12CF12CE881F9810190F081E02D52
:1005900001E0272DA401B501CE0109950E94400973
:1005A0001B012C010E9440096219730984099509F5
:1005B0006C157D058E059F0540F4B501CE010E94A6
:1005C0008902882379F381E004C01F5F6116D8F6A1
:1005D00080E0DF91CF911F910F91FF90EF90DF901E
:1005E000CF90BF90AF909F908F907F906F905F90D3
:1005F0004F903F902F900895EF92FF921F93CF93CB
:10060000DF931F92CDB7DEB77C01DC01ED91FC9149
:100610000688F789E02D698309956981862F8F7790
:100620000E94700280E00E947002182FD701ED91A5
:10063000FC91008CF18DE02DC7010995812F0F9061
:10064000DF91CF911F91FF90EF9008950F931F932B
:10065000CF93DF9300D0CDB7DEB78C01DC01ED91F5
:10066000FC910688F789E02D4A83698309956981A1
:10067000862F80680E9470024A81842F0E94700237
:10068000D801ED91FC91008CF18DE02DC8010F9007
:100690000F90DF91CF911F910F9109941F93CF93EA
:1006A000DF93EC01162F80917701681709F461C080
:1006B000623009F440C070F4662309F444C061302C
:1006C00009F057C061E0CE010E94FC02482F437E32
:1006D00044603FC06330C1F0643009F04AC061E05B
:1006E000CE010E94FC02482F437E4C6061E0CE01A7
:1006F0000E9426038985882381F1E881F981048895
:10070000F589E02D61E014C061E0CE010E94FC0299
:10071000482F437E406161E0CE010E942603898517
:100720008823D9F0E881F9810488F589E02D60E01B
:10073000CE01099512C061E0CE010E94FC02482F53
:10074000437E486006C061E0CE010E94FC02482F53
:10075000437E61E0CE010E942603809177018111E2
:1007600006C067E2CE010E94FC0287FFF6CF10931D
:100770007701DF91CF911F910895CF93DF93EC0123
:10078000603208F06FE168878985882311F06695EB
:10079000688761E1CE010E94FC02482F407E888577
:1007A000482B61E1CE01DF91CF910C9426038F920B
:1007B0009F92AF92BF92CF92DF92EF92FF920F93F0
:1007C0001F93CF93DF931F92CDB7DEB74C016B0120
:1007D000142FB52EF22EA02EDC01ED91FC91028893
:1007E000F389E02D61E0099567E2C4010E94FC02F3
:1007F00087FFFACF40E065E2C4010E9426030F2D77
:100800000E3308F00DE3E11004C0A11004C020E095
:1008100003C020E801C020E4BFEFCB16D10451F0A3
:1008200048F0B6016627737056E0769567955A953D
:10083000E1F7262BF401658176816F3F710521F088
:1008400018F066277370272BD401ED91FC91068870
:10085000F789E02DC4012983099580E80E94700280
:1008600083E0800F0E9470028C2D0E947002F401C0
:1008700085810E9470022981822F0E947002D12EF0
:10088000E12EFB2C8E2D8D19801730F4D7018D9120
:100890007D010E947002F6CFD401ED91FC91008C95
:1008A000F18DE02DC4010995D401ED91FC910288F0
:1008B000F389E02D64E0C40109950E9440096B01B1
:1008C0007C01F40183810E946A0A892BB1F0D40172
:1008D000ED91FC910288F389E02D61E0C4010F9055
:1008E000DF91CF911F910F91FF90EF90DF90CF900C
:1008F000BF90AF909F908F9009940E9440096C190F
:100900007D098E099F09683E734081059105F8F6BF
:10091000D8CFCF93DF93EC0110927601109275013E
:100920001092740110927301109272011092710171
:100930001092700110926F0110926E0110926D0171
:1009400068E20E94FC0282FF0AC06DE3CE010E94B1
:10095000FC02482F44606DE3CE010E94260340E470
:1009600065E2CE010E942603E881F9810288F389BD
:10097000E02D63E0CE01DF91CF910994DF92EF92F9
:10098000FF920F931F93CF93DF93EC018B01E881CC
:10099000F9810288F389E02D61E0099501151105BF
:1009A000E1F0E881F9810688F789E02DCE0109950B
:1009B0008EEB0E9470027801D12CF70181917F01AA
:1009C0000E947002D394F0E1DF12F7CFE881F98141
:1009D000008CF18DE02DCE0109956DE3CE010E94D2
:1009E000FC028E7F91E0012B09F490E0482F492B07
:1009F0006DE3CE01DF91CF911F910F91FF90EF90AA
:100A0000DF900C9426038F929F92AF92BF92CF9269
:100A1000DF92EF92FF920F931F93CF93DF93CDB7A7
:100A2000DEB7AE970FB6F894DEBF0FBECDBF7C0128
:100A30006A01DC0113968C91823021F0833021F41D
:100A400081E003C080E001C08FEFF70184838EE274
:100A50008E010F5F1F4FD801E82F1D92EA95E9F72D
:100A600091E0998334E03A8342E04B8393E09D83A5
:100A70004E833F8340E4488735E039879A8796E084
:100A80009B8793E39C8737E03D8798E09F8799E0B9
:100A9000998B99E19B8B92E49C8B55E25D8B4E8BFD
:100AA00046E24F8B388F38E2398F30E13A8F39E2A6
:100AB0003B8F3CED3C8F8D8F88E88E8F8FE28F8F40
:100AC0008DE288A380E389A337E33BA330E93CA30D
:100AD00038E33DA39EA39CE39FA39FE898A79DE3D3
:100AE00099A792E19AA79FE69BA78CA78FEF8DA766
:100AF0006F3131F06B3231F0663531F489ED05C07C
:100B00008EE403C08CE601C084EE8E876F3141F025
:100B10006B3221F0663521F480E003C080E401C02F
:100B200080EC888B2AA361E0D70112968C910E94F9
:100B3000340A61E0F70182810E94FB090E94E7010B
:100B400080E5D7011C968C931C9781E01D968C93B1
:100B50000E9440094B015C014AEA6FE2C7010E9412
:100B600026036FE2C7010E94FC028A3A59F00E94F4
:100B70004009681979098A099B0962337105810561
:100B8000910550F30E9440094B015C0145E56FE27D
:100B9000C7010E9426036FE2C7010E94FC0285354F
:100BA00059F00E944009681979098A099B09623342
:100BB00071058105910550F3B12CF801EB0DF11D84
:100BC000EB0DF11D60816F3F31F04181C7010E9443
:100BD0002603B394F2CF60E070E0C7010E94BE0428
:100BE000D701ED91FC9111970084F185E02D1996C4
:100BF0006C91C7010995D701ED91FC910288F389A9
:100C0000E02D61E0C70109950E9440094B015C019C
:100C100067E2C7010E94FC0287FD0BC00E944009E9
:100C2000681979098A099B09623371058105910563
:100C300078F30E944009681979098A099B0962338F
:100C400071058105910598F443E050E06EE172E092
:100C5000F70184810E947C08F0926B01E0926A01A6
:100C6000D7011696DC92CE92159781E001C080E004
:100C7000AE960FB6F894DEBF0FBECDBFDF91CF9119
:100C80001F910F91FF90EF90DF90CF90BF90AF90AA
:100C90009F908F900895CF93DF93EC0161110DC069
:100CA00064E2CE010E94FC0290E091958195910949
:100CB00095958795DF91CF91089541E063E20E9479
:100CC000260363E2CE010E94FC0281FFFACFE8CF47
:100CD000CF93DF93EC01809177018330A9F4809169
:100CE0007101811111C060E0CE010E944B06863A6D
:100CF0009F4F54F4E881F9810288F389E02D61E087
:100D0000CE01099581E001C080E0DF91CF91089587
:100D10001F93CF93DF93EC01809177018330D1F45F
:100D200068E2CE010E94FC0282FD20C013C0F0E008
:100D3000E858FE4F1082E881F981008CF18DE02D9A
:100D4000CE010995E881F9810288F389E02D63E0FD
:100D5000CE01099560E0CE010E944B0690936E0192
:100D600080936D01DF91CF911F910895E881F98102
:100D70000288F389E02D61E0CE010995E881F981CF
:100D80000688F789E02DCE01099580E00E94700267
:100D900080E00E947002833408F082E48093710145
:100DA00080E00E94700290E0909373018093720142
:100DB00080E00E94700290E090937501809374012E
:100DC00080E00E947002282F2C7090E4299F9001EF
:100DD00011244091720150917301242B352B3093D3
:100DE000730120937201982F937040917401509178
:100DF0007501592B50937501409374019F81911196
:100E000007C04D815E812417350711F0232B21F493
:100E100090917101933098F410927101E881F981F9
:100E2000008CF18DE02DCE010995E881F9810088D3
:100E3000F189E02DCE01DF91CF911F91099493505C
:100E400090937601982F907890936F01982F9074DB
:100E500090937001E881F9810484F585E02D682F75
:100E6000CE01099510E0E09176011E1708F05FCFE2
:100E700080E00E947002E12FF0E0E858FE4F80838E
:100E80001F5FF1CFCF93DF93EC0180916C0188233A
:100E900029F010926C01CE010E94880680917701A2
:100EA000833071F480917101882389F0E881F981A0
:100EB0000288F389E02D61E0CE01099581E008C048
:100EC000E881F9810088F189E02DCE01099580E063
:100ED000DF91CF9108954F925F926F927F928F92A0
:100EE0009F92AF92BF92EF920F931F93CF93DF9396
:100EF000EC015B014A01122F6DE30E94FC02482FB6
:100F000044606DE3CE010E9426030E9440092B013C
:100F10003C01CE010E9468068823C9F0E881F9816E
:100F20000684F785E02DE12C212FA401B501CE0127
:100F30000995DF91CF911F910F91EF90BF90AF90E6
:100F40009F908F907F906F905F904F9008950E9438
:100F500040096419750986099709683E734081053F
:100F60009105E0F6E881F9810480F581E02DCE015C
:100F70000995CFCF4F925F926F927F928F929F92FF
:100F8000AF92BF92CF92DF92EF920F931F93CF93C6
:100F9000DF93EC014B01142F10927001C09074018B
:100FA000D0907501A0906D01B0906E016DE30E942C
:100FB000FC02482F44606DE3CE010E9426030E948C
:100FC00040092B013C01CE010E946806882329F1CB
:100FD000D0927501C0927401E881F9810684F78589
:100FE000E02DEE24E39400E0212FA401B601CE0110
:100FF0000995B0926E01A0926D01DF91CF911F9182
:101000000F91EF90DF90CF90BF90AF909F908F9017
:101010007F906F905F904F9008950E9440096419EF
:10102000750986099709683E73408105910580F628
:10103000E881F9810480F581E02DCE010995C3CFC7
:10104000CF93DF93EC016987662311F04FE001C075
:101050004AE163E1CE010E9426038985882341F09D
:1010600061E1CE010E94FC02482F4F71406602C030
:101070004885406861E1CE01DF91CF910C94260351
:101080001F93CF93DF93EC01162F662311F04DE5EC
:1010900001C045E56AE5CE010E942603112311F047
:1010A0004CE701C040E76CE5CE01DF91CF911F9185
:1010B0000C9426031F93CF93DF93EC01162FE88146
:1010C000F9810288F389E02D61E0099548E06EE43A
:1010D000CE010E9426036EE4CE010E94FC0282FD36
:1010E000FACF6FE4CE010E94FC021B55181B812F22
:1010F000DF91CF911F9108958230E8F4E82FF0E05E
:10110000EE0FFF1FEA54FE4F71836083813041F080
:10111000809169008C7F842B80936900E89A089500
:1011200080916900440F551F440F551F837F842B06
:1011300080936900E99A08951F920F920FB60F925B
:1011400011242F933F934F935F936F937F938F93CC
:101150009F93AF93BF93EF93FF938091B6019091CC
:10116000B701892B29F0E091B601F091B7010995FB
:10117000FF91EF91BF91AF919F918F917F916F916F
:101180005F914F913F912F910F900FBE0F901F9045
:1011900018951F920F920FB60F9211242F933F9321
:1011A0004F935F936F937F938F939F93AF93BF936F
:1011B000EF93FF938091B8019091B901892B29F0A9
:1011C000E091B801F091B9010995FF91EF91BF91BC
:1011D000AF919F918F917F916F915F914F913F91CF
:1011E0002F910F900FBE0F901F9018951F920F9286
:1011F0000FB60F9211242F933F938F939F93AF932A
:10120000BF938091BB019091BC01A091BD01B091B1
:10121000BE013091BA0126E0230F2D3720F402964B
:10122000A11DB11D05C029E8230F0396A11DB11D05
:101230002093BA018093BB019093BC01A093BD01A0
:10124000B093BE018091BF019091C001A091C101F6
:10125000B091C2010196A11DB11D8093BF01909371
:10126000C001A093C101B093C201BF91AF919F9102
:101270008F913F912F910F900FBE0F901F90189557
:101280002FB7F8946091BB017091BC018091BD01B2
:101290009091BE012FBF08953FB7F8948091BF0190
:1012A0009091C001A091C101B091C20126B5A89B47
:1012B00005C02F3F19F00196A11DB11D3FBF662744
:1012C000782F892F9A2F620F711D811D911D43E088
:1012D000660F771F881F991F4A95D1F70895CF92FF
:1012E000DF92EF92FF92CF93DF936B017C010E941C
:1012F0004C09EB01C114D104E104F10489F00E940E
:10130000700B0E944C096C1B7D0B683E734090F380
:1013100081E0C81AD108E108F108C851DC4FEACFD2
:10132000DF91CF91FF90EF90DF90CF900895789468
:1013300084B5826084BD84B5816084BD85B58260DA
:1013400085BD85B5816085BDEEE6F0E08081816078
:101350008083E1E8F0E01082808182608083808178
:1013600081608083E0E8F0E0808181608083E1EB50
:10137000F0E0808184608083E0EBF0E08081816038
:101380008083EAE7F0E080818460808380818260EE
:10139000808380818E7F80838081806880831092AB
:1013A000C1000895833081F028F4813099F08230B3
:1013B000A1F008958730A9F08830B9F08430D1F4D5
:1013C000809180008F7D03C0809180008F77809313
:1013D0008000089584B58F7702C084B58F7D84BD69
:1013E00008958091B0008F7703C08091B0008F7D09
:1013F0008093B0000895CF93DF9390E0FC01E45810
:10140000FF4F2491FC01E057FF4F8491882349F15D
:1014100090E0880F991FFC01E854FF4FA591B4910B
:1014200082559F4FFC01C591D4919FB7611108C0AF
:10143000F8948C91209582238C93888182230AC012
:10144000623051F4F8948C91322F309583238C9331
:101450008881822B888304C0F8948C91822B8C9392
:101460009FBFDF91CF9108950F931F93CF93DF9389
:101470001F92CDB7DEB7282F30E0F901E859FF4FB2
:101480008491F901E458FF4F1491F901E057FF4F9F
:1014900004910023C9F0882321F069830E94D209B6
:1014A0006981E02FF0E0EE0FFF1FE255FF4FA5919D
:1014B000B4919FB7F8948C91611103C0109581236A
:1014C00001C0812B8C939FBF0F90DF91CF911F9113
:1014D0000F910895CF93DF93282F30E0F901E85959
:1014E000FF4F8491F901E458FF4FD491F901E0577F
:1014F000FF4FC491CC2391F081110E94D209EC2FAF
:10150000F0E0EE0FFF1FEC55FF4FA591B4912C9129
:101510002D2381E090E021F480E002C080E090E0A3
:10152000DF91CF9108951F920F920FB60F92112461
:101530002F938F939F93EF93FF93E091D301F091BB
:10154000D4018081E091D901F091DA0182FD12C0CD
:1015500090818091DC018F5F8F732091DD01821774
:1015600051F0E091DC01F0E0ED53FE4F958F809358
:10157000DC0101C08081FF91EF919F918F912F91AC
:101580000F900FBE0F901F9018951F920F920FB6DD
:101590000F9211242F933F934F935F936F937F93F9
:1015A0008F939F93AF93BF93EF93FF9383EC91E05F
:1015B0000E94AC0BFF91EF91BF91AF919F918F91E2
:1015C0007F916F915F914F913F912F910F900FBE3F
:1015D0000F901F90189583EC91E00E94710B21E011
:1015E000892B09F420E0822F08951092C6011092F1
:1015F000C50188EE93E0A0E0B0E08093C70190932E
:10160000C801A093C901B093CA018FE391E0909300
:10161000C4018093C30185EC90E09093D001809346
:10162000CF0184EC90E09093D2018093D10180ECC3
:1016300090E09093D4018093D30181EC90E090935B
:10164000D6018093D50182EC90E09093D8018093ED
:10165000D70186EC90E09093DA018093D901109243
:10166000DC011092DD011092DE011092DF0108957D
:1016700008950E9497090E94380B0E940A01CEE942
:10168000DBE00E9448012097E1F30E949E0BF9CF16
:10169000CF92DF92EF92FF920F931F93CF93DF933E
:1016A0006C017A01EB01E60EF71E00E010E0CE15AA
:1016B000DF0561F06991D601ED91FC910190F08117
:1016C000E02DC6010995080F191FF1CFC801DF9160
:1016D000CF911F910F91FF90EF90DF90CF900895E1
:1016E0000895FC01818D228D90E0805C9F4F821BCC
:1016F00091098F7399270895FC01918D828D981718
:1017000031F0828DE80FF11D858D90E008958FEF07
:101710009FEF0895FC01918D828D981761F0828D65
:10172000DF01A80FB11D5D968C91928D9F5F9F7315
:10173000928F90E008958FEF9FEF08958BEE9AE0DF
:10174000892B49F080E090E0892B29F00E94EB0A78
:1017500081110C9400000895FC01848DDF01A80F15
:10176000B11DA35ABF4F2C91848D90E001968F73C9
:101770009927848FA689B7892C93A089B1898C91E8
:1017800080648C93938D848D981306C00288F389AE
:10179000E02D80818F7D80830895CF93DF93EC01CE
:1017A000888D8823C9F0EA89FB89808185FD05C081
:1017B000A889B9898C9186FD0FC00FB607FCF5CFBB
:1017C000808185FFF2CFA889B9898C9185FFEDCF03
:1017D000CE010E94AC0BE7CFDF91CF910895CF925D
:1017E000DF92FF920F931F93CF93DF931F92CDB79A
:1017F000DEB76C0181E0D60158968C9358975B96C2
:101800009C915B975C968C915C97981307C050965F
:10181000ED91FC915197808185FD2EC0F601038DDD
:1018200010E00F5F1F4F0F731127F02EF601848D0C
:10183000F81211C00FB607FCF9CFD6015096ED9102
:10184000FC915197808185FFF1CFC60169830E9489
:10185000AC0B6981EBCF838DE80FF11DE35AFF4F8D
:101860006083D6015B960C935B975296ED91FC9149
:101870005397808180620CC0D6015696ED91FC9101
:10188000579760835096ED91FC91519780818064C9
:10189000808381E090E00F90DF91CF911F910F91B5
:1018A000FF90DF90CF900895E89409C097FB3EF435
:1018B00090958095709561957F4F8F4F9F4F99239D
:1018C000A9F0F92F96E9BB279395F695879577951B
:1018D0006795B795F111F8CFFAF4BB0F11F460FFDB
:1018E0001BC06F5F7F4F8F4F9F4F16C0882311F033
:1018F00096E911C0772321F09EE8872F762F05C047
:10190000662371F096E8862F70E060E02AF09A95E1
:10191000660F771F881FDAF7880F9695879597F9D6
:101920000895EE0FFF1F0590F491E02D0994EF92BA
:101930000F931F93CF93DF93E80147FF02C034E179
:1019400001C034E0E42FFF27E7FDF095F7FF03C067
:10195000F195E195F109E32E022F2E2FAE010E94A1
:10196000AC0ECE01DF91CF911F910F91EF900895B2
:10197000AEE0B0E0EEEBFCE00C94B6110D891E89F0
:1019800086E08C831A8309838FEF9FE79E838D8384
:10199000AE01475E5F4F6F89788DCE0101960E9440
:1019A000DA0CEF81F885E00FF11F10822E96E4E04B
:1019B0000C94D211ACE0B0E0E0EEFCE00C94A81185
:1019C0007C016B018A01FC0117821682838181FFF1
:1019D000BDC1CE0101964C01F7019381F60193FD43
:1019E000859193FF81916F01882309F4ABC1853202
:1019F00039F493FD859193FF81916F01853229F42C
:101A0000B70190E00E941811E7CF512C312C20E053
:101A10002032A0F48B3269F030F4803259F08332F6
:101A200069F420612CC08D3239F0803339F42160A3
:101A300026C02260246023C0286021C027FD27C063
:101A400030ED380F3A3078F426FF06C0FAE05F9E9A
:101A5000300D1124532E13C08AE0389E300D11240E
:101A6000332E20620CC08E3221F426FD6BC120641F
:101A700006C08C3611F4206802C0883641F4F601A5
:101A800093FD859193FF81916F018111C1CF982FB3
:101A90009F7D9554933028F40C5F1F4FFFE3F9832B
:101AA0000DC0833631F0833771F0833509F05BC0A8
:101AB00022C0F801808189830E5F1F4F4424439424
:101AC000512C540115C03801F2E06F0E711CF80161
:101AD000A080B18026FF03C0652D70E002C06FEFCB
:101AE0007FEFC5012C870E940D112C0183012C85ED
:101AF0002F77222E17C03801F2E06F0E711CF8010B
:101B0000A080B18026FF03C0652D70E002C06FEF9A
:101B10007FEFC5012C870E9402112C012C852068C3
:101B2000222E830123FC1BC0832D90E0481659060A
:101B3000B0F4B70180E290E00E9418113A94F4CF1B
:101B4000F50127FC859127FE81915F01B70190E0A7
:101B50000E94181131103A94F1E04F1A51084114C3
:101B6000510471F7E5C0843611F0893639F5F80172
:101B700027FF07C060817181828193810C5F1F4FB5
:101B800008C060817181882777FD8095982F0E5F4E
:101B90001F4F2F76B22E97FF09C0909580957095B4
:101BA00061957F4F8F4F9F4F2068B22E2AE030E023
:101BB000A4010E944A11A82EA81844C0853729F410
:101BC0002F7EB22E2AE030E025C0F22FF97FBF2E03
:101BD0008F36C1F018F4883579F0B4C0803719F029
:101BE000883721F0AFC02F2F2061B22EB4FE0DC078
:101BF0008B2D8460B82E09C024FF0AC09F2F9660E9
:101C0000B92E06C028E030E005C020E130E002C077
:101C100020E132E0F801B7FE07C060817181828166
:101C200093810C5F1F4F06C06081718180E090E05E
:101C30000E5F1F4FA4010E944A11A82EA818FB2D69
:101C4000FF77BF2EB6FE0BC02B2D2E7FA51450F4B0
:101C5000B4FE0AC0B2FC08C02B2D2E7E05C07A2C23
:101C60002B2D03C07A2C01C0752C24FF0DC0FE0162
:101C7000EA0DF11D8081803311F4297E09C022FF15
:101C800006C07394739404C0822F867809F073940D
:101C900023FD13C020FF06C05A2C731418F4530CF4
:101CA0005718732C731468F4B70180E290E02C8706
:101CB0000E94181173942C85F5CF731410F4371803
:101CC00001C0312C24FF12C0B70180E390E02C87C3
:101CD0000E9418112C8522FF17C021FF03C088E540
:101CE00090E002C088E790E0B7010CC0822F8678B0
:101CF00059F021FD02C080E201C08BE227FD8DE298
:101D0000B70190E00E941811A51438F4B70180E3E0
:101D100090E00E9418115A94F7CFAA94F401EA0DAA
:101D2000F11D8081B70190E00E941811A110F5CF3C
:101D3000332009F451CEB70180E290E00E941811DF
:101D40003A94F6CFF7018681978102C08FEF9FEF1B
:101D50002C96E2E10C94C4116F927F929F92AF9205
:101D6000BF92CF92DF92EF92FF920F931F93CF9388
:101D7000DF93CDB7DEB729970FB6F894DEBF0FBE5D
:101D8000CDBF6A01B22E102F0C3320F4FF24F39440
:101D9000F00E02C04CE3F42E0F2D27E0AE014F5F92
:101DA0005F4F0E942A107981272F2970213031F04E
:101DB000E1FC06C0E0FC06C060E005C06DE203C0C7
:101DC0006BE201C060E2AE2DA07173FF36C06623E6
:101DD00011F084E001C083E08B1510F4B81A01C043
:101DE000B12CA1110BC0F6018B2D90E2882319F0C4
:101DF00091938150FBCFCB0CD11CB12C662331F0D9
:101E0000F601608396012F5F3F4F6901C60103967B
:101E1000E2FE05C02EE4F601208331E404C02EE684
:101E2000F601208331E631832283FC012B2D30E241
:101E30002223F1F131932150FBCF72FF40C0662382
:101E400011F084E001C083E08B1510F4B81A01C0D2
:101E5000B12CA1110BC0F6018B2D90E2882319F053
:101E600091938150FBCFCB0CD11CB12C662331F068
:101E7000F601608396012F5F3F4F6901C60103960B
:101E8000E2FE07C029E4F60120832EE4218326E444
:101E900006C029E6F60120832EE6218326E622836A
:101EA000FC012B2D30E2222319F031932150FBCF7E
:101EB000FC01EB0DF11D10828EEF9FEFB7C0B1E07A
:101EC000611101C0B0E04B2F50E01816190624F440
:101ED0009C012F5F3F4F02C021E030E0240F351FEF
:101EE000112329F0412F50E04F5F5F4F02C040E0C7
:101EF00050E0420F531F2B2D30E04217530714F4CC
:101F0000B41A01C0B12C2E2D287159F4F6012B2DD5
:101F100030E2222319F031932150FBCFCB0CD11C9E
:101F2000B12CBB2331F0F601608396012F5F3F4F48
:101F30006901A1110BC0F6012B2D30E3222319F00A
:101F400031932150FBCFCB0CD11CB12CF80E0A8160
:101F5000372F3071A32E74FF03C0013309F4FA94B4
:101F60001F142CF42F2D293018F028E001C021E097
:101F7000682F392F97FF02C060E030E0462F532FC3
:101F8000612C712C3EE2932EBC01621B71099B01F6
:101F9000DC01A41BB50BE1E0F0E0EC0FFD1FAE0F80
:101FA000BF1FE12EF12CF194E194F1084F3FFFEFB8
:101FB0005F0731F4F6019082B6016F5F7F4F6B01CE
:101FC000841795074CF02417350734F4BD01660DCE
:101FD000771DFB01118101C010E341505109FFEF52
:101FE0006F1A7F0AB6016F5F7F4F4E155F0524F0B1
:101FF000F60110836B01DACF4817590739F406331D
:1020000020F4053319F4A11001C011E3F601108387
:10201000FB018B2D90E2882319F091938150FBCF27
:10202000FB01EB0DF11D108280E090E029960FB6C8
:10203000F894DEBF0FBECDBFDF91CF911F910F91FE
:10204000FF90EF90DF90CF90BF90AF909F907F90E8
:102050006F900895283008F027E03327DA01990FB0
:10206000311D87FD916000966105710539F432607C
:102070002E5F3D9330E32A95E1F708959F3F30F0BE
:1020800080387105610509F03C5F3C5F3D939130FC
:1020900008F08068911DDF93CF931F930F93FF92F9
:1020A000EF92192F987F9695E92F96959695E90FBF
:1020B000FF27E45EFE4F99273327EE24FF24A70174
:1020C000E70105900894079428F4360FE71EF81EE0
:1020D000491F511D660F771F881F991F0694A1F78E
:1020E0000590079428F4E70EF81E491F561FC11DDE
:1020F000770F881F991F661F0694A1F70590079414
:1021000028F4F80E491F561FC71FD11D880F991FAD
:10211000661F771F0694A1F70590079420F4490FD6
:10212000561FC71FD81F990F661F771F881F069459
:10213000A9F784911095177041F0D695C7955795DA
:102140004795F794E7941A95C1F7E2ECF0E06894AC
:102150001590159135916591959105907FE2739554
:10216000E118F10A430B560BC90BD009C0F7E10C7B
:10217000F11E431F561FC91FD01D7EF4703311F48A
:102180008A95E6CFE894015030F0080F0AF4002752
:10219000021708F4202F2395022F7A3328F079E3D1
:1021A0007D932A95E9F710C07D932A9589F60694C8
:1021B00097956795379517951794E118F10A430B92
:1021C000560BC90BD00998F023957E9173957A33FD
:1021D00008F070E37C932013B8F77E9170617D93D3
:1021E00030F0839571E37D9370E32A95E1F7112434
:1021F000EF90FF900F911F91CF91DF91992787FD6D
:1022000090950895FC010590615070400110D8F739
:10221000809590958E0F9F1F0895FC01615070402E
:1022200001900110D8F7809590958E0F9F1F08950B
:102230000F931F93CF93DF93182F092FEB018B81FF
:1022400081FD03C08FEF9FEF20C082FF10C04E8141
:102250005F812C813D81421753077CF4E881F9812D
:102260009F012F5F3F4F39832883108306C0E88585
:10227000F985812F0995892B29F72E813F812F5FC1
:102280003F4F3F832E83812F902FDF91CF911F915E
:102290000F910895FA01AA27283051F1203181F1D8
:1022A000E8946F936E7F6E5F7F4F8F4F9F4FAF4F5E
:1022B000B1E03ED0B4E03CD0670F781F891F9A1F71
:1022C000A11D680F791F8A1F911DA11D6A0F711D25
:1022D000811D911DA11D20D009F468943F912AE031
:1022E000269F11243019305D3193DEF6CF01089519
:1022F000462F4770405D4193B3E00FD0C9F7F6CF4A
:10230000462F4F70405D4A3318F0495D31FD405211
:10231000419302D0A9F7EACFB4E0A69597958795A7
:1023200077956795BA95C9F7009761057105089586
:102330009B01AC010A2E0694579547953795279532
:10234000BA95C9F7620F731F841F951FA01D0895CA
:102350002F923F924F925F926F927F928F929F92B5
:10236000AF92BF92CF92DF92EF92FF920F931F93A3
:10237000CF93DF93CDB7DEB7CA1BDB0B0FB6F89454
:10238000DEBF0FBECDBF09942A88398848885F8494
:102390006E847D848C849B84AA84B984C884DF8005
:1023A000EE80FD800C811B81AA81B981CE0FD11DE9
:1023B0000FB6F894DEBF0FBECDBFED010895F894BF
:0223C000FFCF4D
:1023C200000060028000544F505345435245545020
:1023D2004153535752440020543A257300000000E1
:1023E200006B07A7024207BA072008BD031D02D7E8
:1023F2000389044E0340084002220200000000EF5D
:0C2402000B480B710B8A0B7C0BCD0B0000
:00000001FF
